 zip

 Timestamp is ffffffff (Sun Feb  7 06:28:15 2106)

 Preferred load address is 10000000

 Start         Length     Name                   Class
 0001:00000000 0000a035H .text$mn                CODE
 0002:00000000 000000f4H .idata$5                DATA
 0002:000000f4 00000004H .00cfg                  DATA
 0002:000000f8 00000004H .CRT$XCA                DATA
 0002:000000fc 00000004H .CRT$XCZ                DATA
 0002:00000100 00000004H .CRT$XIA                DATA
 0002:00000104 00000004H .CRT$XIZ                DATA
 0002:00000108 00000004H .CRT$XPA                DATA
 0002:0000010c 00000004H .CRT$XPZ                DATA
 0002:00000110 00000004H .CRT$XTA                DATA
 0002:00000114 00000004H .CRT$XTZ                DATA
 0002:00000118 00000000H .gfids$y                DATA
 0002:00000118 00004700H .rdata                  DATA
 0002:00004818 00000004H .rdata$sxdata           DATA
 0002:0000481c 00000280H .rdata$zzzdbg           DATA
 0002:00004a9c 00000004H .rtc$IAA                DATA
 0002:00004aa0 00000004H .rtc$IZZ                DATA
 0002:00004aa4 00000004H .rtc$TAA                DATA
 0002:00004aa8 00000008H .rtc$TZZ                DATA
 0002:00004ab0 00000090H .xdata$x                DATA
 0002:00004b40 000006c8H .edata                  DATA
 0002:00005208 000000a0H .idata$2                DATA
 0002:000052a8 00000014H .idata$3                DATA
 0002:000052bc 000000f4H .idata$4                DATA
 0002:000053b0 000004d8H .idata$6                DATA
 0003:00000000 00000028H .data                   DATA
 0003:00000028 00000384H .bss                    DATA
 0004:00000000 00000060H .rsrc$01                DATA
 0004:00000060 00000310H .rsrc$02                DATA

  Address         Publics by Value              Rva+Base       Lib:Object

 0000:00000000       ___arm64x_native_entrypoint 00000000     <absolute>
 0000:00000000       ___guard_longjmp_table     00000000     <absolute>
 0000:00000000       ___guard_fids_count        00000000     <absolute>
 0000:00000000       ___x64_code_ranges_to_entry_points 00000000     <absolute>
 0000:00000000       ___hybrid_code_map         00000000     <absolute>
 0000:00000000       ___guard_eh_cont_count     00000000     <absolute>
 0000:00000000       ___arm64x_redirection_metadata 00000000     <absolute>
 0000:00000000       ___guard_fids_table        00000000     <absolute>
 0000:00000000       ___arm64x_extra_rfe_table_size 00000000     <absolute>
 0000:00000000       ___arm64x_extra_rfe_table  00000000     <absolute>
 0000:00000000       ___guard_iat_count         00000000     <absolute>
 0000:00000000       ___guard_iat_table         00000000     <absolute>
 0000:00000000       ___dynamic_value_reloc_table 00000000     <absolute>
 0000:00000000       ___guard_longjmp_count     00000000     <absolute>
 0000:00000000       ___hybrid_code_map_count   00000000     <absolute>
 0000:00000000       ___enclave_config          00000000     <absolute>
 0000:00000000       ___hybrid_auxiliary_iat    00000000     <absolute>
 0000:00000000       ___arm64x_redirection_metadata_count 00000000     <absolute>
 0000:00000000       ___guard_eh_cont_table     00000000     <absolute>
 0000:00000000       ___volatile_metadata       00000000     <absolute>
 0000:00000000       ___AbsoluteZero            00000000     <absolute>
 0000:00000000       ___x64_code_ranges_to_entry_points_count 00000000     <absolute>
 0000:00000001       ___safe_se_handler_count   00000001     <absolute>
 0000:00000100       ___guard_flags             00000100     <absolute>
 0000:00000000       ___ImageBase               10000000     <linker-defined>
 0001:00000000       _Java_java_util_zip_Adler32_update@16 10001000 f   Adler32.obj
 0001:0000001e       _Java_java_util_zip_Adler32_updateByteBuffer@28 1000101e f   Adler32.obj
 0001:00000045       _Java_java_util_zip_Adler32_updateBytes@24 10001045 f   Adler32.obj
 0001:00000095       _Java_java_util_zip_CRC32_update@16 10001095 f   CRC32.obj
 0001:000000b3       _Java_java_util_zip_CRC32_updateByteBuffer0@28 100010b3 f   CRC32.obj
 0001:000000da       _Java_java_util_zip_CRC32_updateBytes0@24 100010da f   CRC32.obj
 0001:0000012a       _ZIP_CRC32                 1000112a f   CRC32.obj
 0001:0000012f       _Java_java_util_zip_Deflater_deflateBufferBuffer@48 1000112f f   Deflater.obj
 0001:00000171       _Java_java_util_zip_Deflater_deflateBufferBytes@48 10001171 f   Deflater.obj
 0001:000001ff       _Java_java_util_zip_Deflater_deflateBytesBuffer@48 100011ff f   Deflater.obj
 0001:0000028d       _Java_java_util_zip_Deflater_deflateBytesBytes@48 1000128d f   Deflater.obj
 0001:00000367       _Java_java_util_zip_Deflater_end@16 10001367 f   Deflater.obj
 0001:00000394       _Java_java_util_zip_Inflater_getAdler@16 10001394 f   Inflater.obj
 0001:00000394       _Java_java_util_zip_Deflater_getAdler@16 10001394 f   Deflater.obj
 0001:0000039e       _Java_java_util_zip_Deflater_init@20 1000139e f   Deflater.obj
 0001:0000044e       _Java_java_util_zip_Deflater_reset@16 1000144e f   Deflater.obj
 0001:0000046d       _Java_java_util_zip_Deflater_setDictionary@28 1000146d f   Deflater.obj
 0001:000004c6       _Java_java_util_zip_Deflater_setDictionaryBuffer@28 100014c6 f   Deflater.obj
 0001:00000636       _Java_java_util_zip_Inflater_end@16 10001636 f   Inflater.obj
 0001:00000660       _Java_java_util_zip_Inflater_inflateBufferBuffer@40 10001660 f   Inflater.obj
 0001:00000699       _Java_java_util_zip_Inflater_inflateBufferBytes@40 10001699 f   Inflater.obj
 0001:00000720       _Java_java_util_zip_Inflater_inflateBytesBuffer@40 10001720 f   Inflater.obj
 0001:000007a7       _Java_java_util_zip_Inflater_inflateBytesBytes@40 100017a7 f   Inflater.obj
 0001:00000878       _Java_java_util_zip_Inflater_init@12 10001878 f   Inflater.obj
 0001:0000090d       _Java_java_util_zip_Inflater_initIDs@8 1000190d f   Inflater.obj
 0001:0000094d       _Java_java_util_zip_Inflater_reset@16 1000194d f   Inflater.obj
 0001:00000969       _Java_java_util_zip_Inflater_setDictionary@28 10001969 f   Inflater.obj
 0001:000009c2       _Java_java_util_zip_Inflater_setDictionaryBuffer@28 100019c2 f   Inflater.obj
 0001:00001665       _deflate                   10002665 f   deflate.obj
 0001:00001ec8       _deflateBound              10002ec8 f   deflate.obj
 0001:00001f98       _deflateEnd                10002f98 f   deflate.obj
 0001:0000201b       _deflateInit2_             1000301b f   deflate.obj
 0001:00002220       _deflateParams             10003220 f   deflate.obj
 0001:00002345       _deflateReset              10003345 f   deflate.obj
 0001:00002366       _deflateResetKeep          10003366 f   deflate.obj
 0001:000023ec       _deflateSetDictionary      100033ec f   deflate.obj
 0001:00002568       _deflateSetHeader          10003568 f   deflate.obj
 0001:00002ea7       ___local_stdio_printf_options 10003ea7 f i gzlib.obj
 0001:00002ead       _inflate_fast              10003ead f   inffast.obj
 0001:000032ca       _inflate                   100042ca f   inflate.obj
 0001:000049ba       _inflateEnd                100059ba f   inflate.obj
 0001:000049f6       _inflateInit2_             100059f6 f   inflate.obj
 0001:00004a9c       _inflateReset              10005a9c f   inflate.obj
 0001:00004ac5       _inflateReset2             10005ac5 f   inflate.obj
 0001:00004b38       _inflateResetKeep          10005b38 f   inflate.obj
 0001:00004bab       _inflateSetDictionary      10005bab f   inflate.obj
 0001:00004d27       _inflate_table             10005d27 f   inftrees.obj
 0001:00005144       __tr_align                 10006144 f   trees.obj
 0001:00005209       __tr_flush_bits            10006209 f   trees.obj
 0001:0000520e       __tr_flush_block           1000620e f   trees.obj
 0001:0000541f       __tr_init                  1000641f f   trees.obj
 0001:0000547c       __tr_stored_block          1000647c f   trees.obj
 0001:000068aa       _adler32                   100078aa f   zadler32.obj
 0001:000068af       _adler32_z                 100078af f   zadler32.obj
 0001:00006aec       _crc32                     10007aec f   zcrc32.obj
 0001:00006d92       _InflateFully              10007d92 f   zip_util.obj
 0001:00007089       _ZIP_Close                 10008089 f   zip_util.obj
 0001:000070ea       _ZIP_FindEntry             100080ea f   zip_util.obj
 0001:0000711e       _ZIP_FreeEntry             1000811e f   zip_util.obj
 0001:0000716c       _ZIP_GZip_Fully            1000816c f   zip_util.obj
 0001:0000723a       _ZIP_GZip_InitParams       1000823a f   zip_util.obj
 0001:0000729c       _ZIP_GetEntry              1000829c f   zip_util.obj
 0001:000072c8       _ZIP_GetEntry2             100082c8 f   zip_util.obj
 0001:000073d0       _ZIP_GetEntryDataOffset    100083d0 f   zip_util.obj
 0001:000074b5       _ZIP_GetNextEntry          100084b5 f   zip_util.obj
 0001:000074f5       _ZIP_Get_From_Cache        100084f5 f   zip_util.obj
 0001:000075ee       _ZIP_InflateFully          100085ee f   zip_util.obj
 0001:000076a9       _ZIP_Open                  100086a9 f   zip_util.obj
 0001:000076e3       _ZIP_Open_Generic          100086e3 f   zip_util.obj
 0001:00007731       _ZIP_Put_In_Cache          10008731 f   zip_util.obj
 0001:00007752       _ZIP_Put_In_Cache0         10008752 f   zip_util.obj
 0001:0000793c       _ZIP_Read                  1000893c f   zip_util.obj
 0001:00007a5c       _ZIP_ReadEntry             10008a5c f   zip_util.obj
 0001:00007d4a       _equals                    10008d4a f   zip_util.obj
 0001:0000900c       _zcfree                    1000a00c f   zutil.obj
 0001:000091a5       @_guard_check_icall_nop@4  1000a1a5 f   MSVCRT:guard_support.obj
 0001:000091a8       _zcalloc                   1000a1a8 f   zutil.obj
 0001:000091ba       _jio_fprintf               1000a1ba f   jvm:jvm.dll
 0001:000091c0       _JVM_NativePath@4          1000a1c0 f   jvm:jvm.dll
 0001:000091c6       _JVM_RawMonitorCreate@0    1000a1c6 f   jvm:jvm.dll
 0001:000091cc       _JVM_RawMonitorDestroy@4   1000a1cc f   jvm:jvm.dll
 0001:000091d2       _JVM_RawMonitorEnter@4     1000a1d2 f   jvm:jvm.dll
 0001:000091d8       _JVM_RawMonitorExit@4      1000a1d8 f   jvm:jvm.dll
 0001:000091de       _JNU_ThrowOutOfMemoryError@8 1000a1de f   java:java.dll
 0001:000091e4       _JNU_ThrowIllegalArgumentException@8 1000a1e4 f   java:java.dll
 0001:000091ea       _JNU_ThrowInternalError@8  1000a1ea f   java:java.dll
 0001:000091f0       _JNU_ThrowByName@12        1000a1f0 f   java:java.dll
 0001:000091f6       _getLastErrorString@8      1000a1f6 f   java:java.dll
 0001:000091fc       _getErrorString@12         1000a1fc f   java:java.dll
 0001:00009202       _getPrefixed               1000a202 f   java:java.dll
 0001:00009208       _handleRead                1000a208 f   java:java.dll
 0001:0000920e       _handleLseek@20            1000a20e f   java:java.dll
 0001:00009214       @__security_check_cookie@4 1000a214 f   MSVCRT:secchk.obj
 0001:00009230       __allrem                   1000a230 f   MSVCRT:llrem.obj
 0001:000092f0       __chkstk                   1000a2f0 f   MSVCRT:chkstk.obj
 0001:000092f0       __alloca_probe             1000a2f0 f   MSVCRT:chkstk.obj
 0001:0000965d       __DllMainCRTStartup@12     1000a65d f   MSVCRT:dll_dllmain.obj
 0001:00009680       ___raise_securityfailure   1000a680 f   MSVCRT:gs_report.obj
 0001:000096a8       ___report_gsfailure        1000a6a8 f   MSVCRT:gs_report.obj
 0001:000097ee       ___security_init_cookie    1000a7ee f   MSVCRT:gs_support.obj
 0001:00009839       _DllMain@12                1000a839 f   MSVCRT:dll_dllmain_stub.obj
 0001:0000985b       ?__scrt_initialize_type_info@@YAXXZ 1000a85b f   MSVCRT:tncleanup.obj
 0001:00009867       ?__scrt_uninitialize_type_info@@YAXXZ 1000a867 f   MSVCRT:tncleanup.obj
 0001:00009873       ___local_stdio_scanf_options 1000a873 f i MSVCRT:default_local_stdio_options.obj
 0001:00009879       ___scrt_initialize_default_local_stdio_options 1000a879 f   MSVCRT:default_local_stdio_options.obj
 0001:000098da       ___scrt_acquire_startup_lock 1000a8da f   MSVCRT:utility.obj
 0001:0000990c       ___scrt_dllmain_after_initialize_c 1000a90c f   MSVCRT:utility.obj
 0001:00009937       ___scrt_dllmain_before_initialize_c 1000a937 f   MSVCRT:utility.obj
 0001:00009945       ___scrt_dllmain_crt_thread_attach 1000a945 f   MSVCRT:utility.obj
 0001:00009964       ___scrt_dllmain_crt_thread_detach 1000a964 f   MSVCRT:utility.obj
 0001:00009971       ___scrt_dllmain_exception_filter 1000a971 f   MSVCRT:utility.obj
 0001:000099a5       ___scrt_dllmain_uninitialize_c 1000a9a5 f   MSVCRT:utility.obj
 0001:000099c8       ___scrt_dllmain_uninitialize_critical 1000a9c8 f   MSVCRT:utility.obj
 0001:000099d5       ___scrt_initialize_crt     1000a9d5 f   MSVCRT:utility.obj
 0001:00009a0e       ___scrt_initialize_onexit_tables 1000aa0e f   MSVCRT:utility.obj
 0001:00009a95       ___scrt_is_nonwritable_in_current_image 1000aa95 f   MSVCRT:utility.obj
 0001:00009b29       ___scrt_release_startup_lock 1000ab29 f   MSVCRT:utility.obj
 0001:00009b46       ___scrt_uninitialize_crt   1000ab46 f   MSVCRT:utility.obj
 0001:00009b6e       ___scrt_get_dyn_tls_init_callback 1000ab6e f   MSVCRT:dyn_tls_init.obj
 0001:00009b74       ___scrt_fastfail           1000ab74 f   MSVCRT:utility_desktop.obj
 0001:00009c8e       __crt_debugger_hook        1000ac8e f   MSVCRT:utility_desktop.obj
 0001:00009c96       __RTC_Initialize           1000ac96 f   MSVCRT:initsect.obj
 0001:00009cc2       __RTC_Terminate            1000acc2 f   MSVCRT:initsect.obj
 0001:00009cf0       __SEH_prolog4              1000acf0 f   MSVCRT:sehprolg4.obj
 0001:00009d34       __SEH_epilog4              1000ad34 f   MSVCRT:sehprolg4.obj
 0001:00009d48       __except_handler4          1000ad48 f   MSVCRT:chandler4gs.obj
 0001:00009d77       ___isa_available_init      1000ad77 f   MSVCRT:cpu_disp.obj
 0001:00009f47       __get_startup_argv_mode    1000af47 f   MSVCRT:argv_mode.obj
 0001:00009f4b       ___scrt_is_ucrt_dll_in_use 1000af4b f   MSVCRT:ucrt_detection.obj
 0001:00009f57       _IsProcessorFeaturePresent@4 1000af57 f   kernel32:KERNEL32.dll
 0001:00009f5d       _memcpy                    1000af5d f   vcruntime:VCRUNTIME140.dll
 0001:00009f63       _memset                    1000af63 f   vcruntime:VCRUNTIME140.dll
 0001:00009f69       ___std_type_info_destroy_list 1000af69 f   vcruntime:VCRUNTIME140.dll
 0001:00009f6f       __except_handler4_common   1000af6f f   vcruntime:VCRUNTIME140.dll
 0001:00009f75       _strlen                    1000af75 f   ucrt:api-ms-win-crt-string-l1-1-0.dll
 0001:00009f7b       _strcmp                    1000af7b f   ucrt:api-ms-win-crt-string-l1-1-0.dll
 0001:00009f81       _strcpy                    1000af81 f   ucrt:api-ms-win-crt-string-l1-1-0.dll
 0001:00009f87       __initterm                 1000af87 f   ucrt:api-ms-win-crt-runtime-l1-1-0.dll
 0001:00009f8d       __initterm_e               1000af8d f   ucrt:api-ms-win-crt-runtime-l1-1-0.dll
 0001:00009f93       __seh_filter_dll           1000af93 f   ucrt:api-ms-win-crt-runtime-l1-1-0.dll
 0001:00009f99       __configure_narrow_argv    1000af99 f   ucrt:api-ms-win-crt-runtime-l1-1-0.dll
 0001:00009f9f       __initialize_narrow_environment 1000af9f f   ucrt:api-ms-win-crt-runtime-l1-1-0.dll
 0001:00009fa5       __initialize_onexit_table  1000afa5 f   ucrt:api-ms-win-crt-runtime-l1-1-0.dll
 0001:00009fab       __execute_onexit_table     1000afab f   ucrt:api-ms-win-crt-runtime-l1-1-0.dll
 0001:00009fb1       __cexit                    1000afb1 f   ucrt:api-ms-win-crt-runtime-l1-1-0.dll
 0001:00009fb7       ___vcrt_initialize         1000afb7 f   MSVCRT:ucrt_stubs.obj
 0001:00009fb7       ___vcrt_thread_attach      1000afb7 f   MSVCRT:ucrt_stubs.obj
 0001:00009fb7       ___scrt_stub_for_acrt_thread_detach 1000afb7 f   MSVCRT:ucrt_stubs.obj
 0001:00009fb7       ___scrt_stub_for_acrt_thread_attach 1000afb7 f   MSVCRT:ucrt_stubs.obj
 0001:00009fb7       ___acrt_uninitialize       1000afb7 f   MSVCRT:ucrt_stubs.obj
 0001:00009fb7       ___acrt_thread_detach      1000afb7 f   MSVCRT:ucrt_stubs.obj
 0001:00009fb7       ___acrt_thread_attach      1000afb7 f   MSVCRT:ucrt_stubs.obj
 0001:00009fb7       ___scrt_stub_for_acrt_uninitialize 1000afb7 f   MSVCRT:ucrt_stubs.obj
 0001:00009fb7       ___vcrt_uninitialize       1000afb7 f   MSVCRT:ucrt_stubs.obj
 0001:00009fb7       ___scrt_stub_for_acrt_initialize 1000afb7 f   MSVCRT:ucrt_stubs.obj
 0001:00009fb7       ___vcrt_thread_detach      1000afb7 f   MSVCRT:ucrt_stubs.obj
 0001:00009fb7       ___acrt_initialize         1000afb7 f   MSVCRT:ucrt_stubs.obj
 0001:00009fb7       ___vcrt_uninitialize_critical 1000afb7 f   MSVCRT:ucrt_stubs.obj
 0001:00009fb7       ___scrt_stub_for_acrt_uninitialize_critical 1000afb7 f   MSVCRT:ucrt_stubs.obj
 0001:00009fb7       ___acrt_uninitialize_critical 1000afb7 f   MSVCRT:ucrt_stubs.obj
 0001:00009fba       ___scrt_stub_for_is_c_termination_complete 1000afba f   MSVCRT:ucrt_stubs.obj
 0001:00009fba       __is_c_termination_complete 1000afba f   MSVCRT:ucrt_stubs.obj
 0001:00009fbd       __filter_x86_sse2_floating_point_exception 1000afbd f   MSVCRT:x86_exception_filter.obj
 0001:00009fbd       __filter_x86_sse2_floating_point_exception_default 1000afbd f   MSVCRT:x86_exception_filter.obj
 0002:00000000       __imp__TerminateProcess@8  1000c000     kernel32:KERNEL32.dll
 0002:00000004       __imp__GetCurrentProcess@0 1000c004     kernel32:KERNEL32.dll
 0002:00000008       __imp__SetUnhandledExceptionFilter@4 1000c008     kernel32:KERNEL32.dll
 0002:0000000c       __imp__UnhandledExceptionFilter@4 1000c00c     kernel32:KERNEL32.dll
 0002:00000010       __imp__MultiByteToWideChar@24 1000c010     kernel32:KERNEL32.dll
 0002:00000014       __imp__CloseHandle@4       1000c014     kernel32:KERNEL32.dll
 0002:00000018       __imp__CreateFileW@28      1000c018     kernel32:KERNEL32.dll
 0002:0000001c       __imp__CreateFileA@28      1000c01c     kernel32:KERNEL32.dll
 0002:00000020       __imp__IsDebuggerPresent@0 1000c020     kernel32:KERNEL32.dll
 0002:00000024       __imp__InitializeSListHead@4 1000c024     kernel32:KERNEL32.dll
 0002:00000028       __imp__DisableThreadLibraryCalls@4 1000c028     kernel32:KERNEL32.dll
 0002:0000002c       __imp__GetSystemTimeAsFileTime@4 1000c02c     kernel32:KERNEL32.dll
 0002:00000030       __imp__GetCurrentThreadId@0 1000c030     kernel32:KERNEL32.dll
 0002:00000034       __imp__GetCurrentProcessId@0 1000c034     kernel32:KERNEL32.dll
 0002:00000038       __imp__QueryPerformanceCounter@4 1000c038     kernel32:KERNEL32.dll
 0002:0000003c       __imp__IsProcessorFeaturePresent@4 1000c03c     kernel32:KERNEL32.dll
 0002:00000040       \177KERNEL32_NULL_THUNK_DATA 1000c040     kernel32:KERNEL32.dll
 0002:00000044       __imp__memcpy              1000c044     vcruntime:VCRUNTIME140.dll
 0002:00000048       __imp___except_handler4_common 1000c048     vcruntime:VCRUNTIME140.dll
 0002:0000004c       __imp____std_type_info_destroy_list 1000c04c     vcruntime:VCRUNTIME140.dll
 0002:00000050       __imp__memset              1000c050     vcruntime:VCRUNTIME140.dll
 0002:00000054       \177VCRUNTIME140_NULL_THUNK_DATA 1000c054     vcruntime:VCRUNTIME140.dll
 0002:00000058       __imp__calloc              1000c058     ucrt:api-ms-win-crt-heap-l1-1-0.dll
 0002:0000005c       __imp__realloc             1000c05c     ucrt:api-ms-win-crt-heap-l1-1-0.dll
 0002:00000060       __imp__malloc              1000c060     ucrt:api-ms-win-crt-heap-l1-1-0.dll
 0002:00000064       __imp__free                1000c064     ucrt:api-ms-win-crt-heap-l1-1-0.dll
 0002:00000068       \177api-ms-win-crt-heap-l1-1-0_NULL_THUNK_DATA 1000c068     ucrt:api-ms-win-crt-heap-l1-1-0.dll
 0002:0000006c       __imp___execute_onexit_table 1000c06c     ucrt:api-ms-win-crt-runtime-l1-1-0.dll
 0002:00000070       __imp___initialize_narrow_environment 1000c070     ucrt:api-ms-win-crt-runtime-l1-1-0.dll
 0002:00000074       __imp___cexit              1000c074     ucrt:api-ms-win-crt-runtime-l1-1-0.dll
 0002:00000078       __imp___configure_narrow_argv 1000c078     ucrt:api-ms-win-crt-runtime-l1-1-0.dll
 0002:0000007c       __imp___initialize_onexit_table 1000c07c     ucrt:api-ms-win-crt-runtime-l1-1-0.dll
 0002:00000080       __imp___seh_filter_dll     1000c080     ucrt:api-ms-win-crt-runtime-l1-1-0.dll
 0002:00000084       __imp___initterm_e         1000c084     ucrt:api-ms-win-crt-runtime-l1-1-0.dll
 0002:00000088       __imp___initterm           1000c088     ucrt:api-ms-win-crt-runtime-l1-1-0.dll
 0002:0000008c       __imp___errno              1000c08c     ucrt:api-ms-win-crt-runtime-l1-1-0.dll
 0002:00000090       \177api-ms-win-crt-runtime-l1-1-0_NULL_THUNK_DATA 1000c090     ucrt:api-ms-win-crt-runtime-l1-1-0.dll
 0002:00000094       __imp____acrt_iob_func     1000c094     ucrt:api-ms-win-crt-stdio-l1-1-0.dll
 0002:00000098       \177api-ms-win-crt-stdio-l1-1-0_NULL_THUNK_DATA 1000c098     ucrt:api-ms-win-crt-stdio-l1-1-0.dll
 0002:0000009c       __imp__strdup              1000c09c     ucrt:api-ms-win-crt-string-l1-1-0.dll
 0002:0000009c       __imp___strdup             1000c09c     ucrt:api-ms-win-crt-string-l1-1-0.dll
 0002:000000a0       __imp__strlen              1000c0a0     ucrt:api-ms-win-crt-string-l1-1-0.dll
 0002:000000a4       __imp__strcmp              1000c0a4     ucrt:api-ms-win-crt-string-l1-1-0.dll
 0002:000000a8       __imp__strcpy              1000c0a8     ucrt:api-ms-win-crt-string-l1-1-0.dll
 0002:000000ac       \177api-ms-win-crt-string-l1-1-0_NULL_THUNK_DATA 1000c0ac     ucrt:api-ms-win-crt-string-l1-1-0.dll
 0002:000000b0       __imp__JNU_ThrowInternalError@8 1000c0b0     java:java.dll
 0002:000000b4       __imp__JNU_ThrowIllegalArgumentException@8 1000c0b4     java:java.dll
 0002:000000b8       __imp__JNU_ThrowOutOfMemoryError@8 1000c0b8     java:java.dll
 0002:000000bc       __imp__getLastErrorString@8 1000c0bc     java:java.dll
 0002:000000c0       __imp__getPrefixed         1000c0c0     java:java.dll
 0002:000000c4       __imp__handleRead          1000c0c4     java:java.dll
 0002:000000c8       __imp__handleLseek@20      1000c0c8     java:java.dll
 0002:000000cc       __imp__JNU_ThrowByName@12  1000c0cc     java:java.dll
 0002:000000d0       __imp__getErrorString@12   1000c0d0     java:java.dll
 0002:000000d4       \177java_NULL_THUNK_DATA   1000c0d4     java:java.dll
 0002:000000d8       __imp__JVM_RawMonitorExit@4 1000c0d8     jvm:jvm.dll
 0002:000000dc       __imp__JVM_RawMonitorCreate@0 1000c0dc     jvm:jvm.dll
 0002:000000e0       __imp__jio_fprintf         1000c0e0     jvm:jvm.dll
 0002:000000e4       __imp__JVM_RawMonitorEnter@4 1000c0e4     jvm:jvm.dll
 0002:000000e8       __imp__JVM_NativePath@4    1000c0e8     jvm:jvm.dll
 0002:000000ec       __imp__JVM_RawMonitorDestroy@4 1000c0ec     jvm:jvm.dll
 0002:000000f0       \177jvm_NULL_THUNK_DATA    1000c0f0     jvm:jvm.dll
 0002:000000f4       ___guard_check_icall_fptr  1000c0f4     MSVCRT:guard_support.obj
 0002:000000f8       ___xc_a                    1000c0f8     MSVCRT:initializers.obj
 0002:000000fc       ___xc_z                    1000c0fc     MSVCRT:initializers.obj
 0002:00000100       ___xi_a                    1000c100     MSVCRT:initializers.obj
 0002:00000104       ___xi_z                    1000c104     MSVCRT:initializers.obj
 0002:00000108       ___xp_a                    1000c108     MSVCRT:initializers.obj
 0002:0000010c       ___xp_z                    1000c10c     MSVCRT:initializers.obj
 0002:00000110       ___xt_a                    1000c110     MSVCRT:initializers.obj
 0002:00000114       ___xt_z                    1000c114     MSVCRT:initializers.obj
 0002:00000118       ??_C@_06CJNJFBNP@1?42?411@ 1000c118     Deflater.obj
 0002:00000120       ??_C@_0FE@LGLGPGLE@zlib?5returned?5Z_VERSION_ERROR?3?5@ 1000c120     Deflater.obj
 0002:00000174       ??_C@_0CI@GPICINMP@unknown?5error?5initializing?5zlib@ 1000c174     Deflater.obj
 0002:0000019c       ??_C@_0CK@JIKCJEKE@unknown?5error?5in?5checkSetDictio@ 1000c19c     Deflater.obj
 0002:000001c8       ??_C@_0DE@MNJNEBHM@unknown?5error?5in?5checkDeflateSt@ 1000c1c8     Deflater.obj
 0002:000001fc       ??_C@_0CE@HKIKJBPI@unknown?5error?5in?5checkDeflateSt@ 1000c1fc     Deflater.obj
 0002:00000220       ??_C@_0BE@IEHJKMAD@deflateReset?5failed@ 1000c220     Deflater.obj
 0002:00000234       ??_C@_0BC@FEOAJDAI@deflateEnd?5failed@ 1000c234     Deflater.obj
 0002:00000248       ??_C@_01JPJNBJEM@I@        1000c248     Inflater.obj
 0002:0000024c       ??_C@_0O@KDFPFIBD@inputConsumed@ 1000c24c     Inflater.obj
 0002:0000025c       ??_C@_0P@HBJOMJPA@outputConsumed@ 1000c25c     Inflater.obj
 0002:0000026c       ??_C@_0CF@BEGCBKMP@inflateInit2?5returned?5Z_STREAM_@ 1000c26c     Inflater.obj
 0002:00000294       ??_C@_0CC@MDBAKBOC@java?1util?1zip?1DataFormatExcepti@ 1000c294     Inflater.obj
 0002:000002b8       _deflate_copyright         1000c2b8     deflate.obj
 0002:0000037f       ??_C@_00CNPNBAHC@@         1000c37f     gzlib.obj
 0002:00000c28       ??_C@_0BD@PJCBIDD@invalid?5block?5type@ 1000cc28     infback.obj
 0002:00000c3c       ??_C@_0BN@LGAADGOK@invalid?5stored?5block?5lengths@ 1000cc3c     infback.obj
 0002:00000c5c       ??_C@_0CE@GMIGFPBB@too?5many?5length?5or?5distance?5sym@ 1000cc5c     infback.obj
 0002:00000c80       ??_C@_0BJ@HDEPPGOH@invalid?5code?5lengths?5set@ 1000cc80     infback.obj
 0002:00000c9c       ??_C@_0BK@BMMPFBBH@invalid?5bit?5length?5repeat@ 1000cc9c     infback.obj
 0002:00000cb8       ??_C@_0CF@DGDMADCD@invalid?5code?5?9?9?5missing?5end?9of?9@ 1000ccb8     infback.obj
 0002:00000ce0       ??_C@_0BM@IIMGAINC@invalid?5literal?1lengths?5set@ 1000cce0     infback.obj
 0002:00000cfc       ??_C@_0BG@GMDFCBGP@invalid?5distances?5set@ 1000ccfc     infback.obj
 0002:00000d14       ??_C@_0BM@FFFLPBBC@invalid?5literal?1length?5code@ 1000cd14     infback.obj
 0002:00000d30       ??_C@_0BG@LBKINIKP@invalid?5distance?5code@ 1000cd30     infback.obj
 0002:00000d48       ??_C@_0BO@ECPMAOGG@invalid?5distance?5too?5far?5back@ 1000cd48     infback.obj
 0002:00001610       ??_C@_0BH@LIBMMIGA@incorrect?5header?5check@ 1000d610     inflate.obj
 0002:00001628       ??_C@_0BL@IHKGDAEE@unknown?5compression?5method@ 1000d628     inflate.obj
 0002:00001644       ??_C@_0BE@EMOGCLGO@invalid?5window?5size@ 1000d644     inflate.obj
 0002:00001658       ??_C@_0BJ@BLBBCOMO@unknown?5header?5flags?5set@ 1000d658     inflate.obj
 0002:00001674       ??_C@_0BE@GONKLEPM@header?5crc?5mismatch@ 1000d674     inflate.obj
 0002:00001688       ??_C@_0BF@MEIGEHBE@incorrect?5data?5check@ 1000d688     inflate.obj
 0002:000016a0       ??_C@_0BH@FGKKJGOC@incorrect?5length?5check@ 1000d6a0     inflate.obj
 0002:000016b8       _inflate_copyright         1000d6b8     inftrees.obj
 0002:000017e8       __length_code              1000d7e8     trees.obj
 0002:000018e8       __dist_code                1000d8e8     trees.obj
 0002:00004268       ??_C@_09CDDFBEOB@META?9INF?1@ 10010268     zip_util.obj
 0002:00004274       ??_C@_0DA@LDHLKKMA@invalid?5END?5header?5?$CIbad?5central@ 10010274     zip_util.obj
 0002:000042a4       ??_C@_0DC@HNGNGCGO@invalid?5END?5header?5?$CIbad?5central@ 100102a4     zip_util.obj
 0002:000042d8       ??_C@_0CD@OGNDFFDB@invalid?5CEN?5header?5?$CIbad?5signatu@ 100102d8     zip_util.obj
 0002:000042fc       ??_C@_0CF@JMIBKLMP@invalid?5CEN?5header?5?$CIencrypted?5e@ 100102fc     zip_util.obj
 0002:00004324       ??_C@_0CM@OFBGAGKC@invalid?5CEN?5header?5?$CIbad?5compres@ 10010324     zip_util.obj
 0002:00004350       ??_C@_0CF@EDCPNMDL@invalid?5CEN?5header?5?$CIbad?5header?5@ 10010350     zip_util.obj
 0002:00004378       ??_C@_0BH@LJLKODMB@zip?5file?5name?5too?5long@ 10010378     zip_util.obj
 0002:00004390       ??_C@_0BC@FKAFCEIB@zip?5file?5is?5empty@ 10010390     zip_util.obj
 0002:000043a4       ??_C@_0BE@LOIOAONC@Zip?5file?5open?5error@ 100103a4     zip_util.obj
 0002:000043b8       ??_C@_0BH@LBOCJMDB@error?5reading?5zip?5file@ 100103b8     zip_util.obj
 0002:000043d0       ??_C@_0CD@MENKOKKM@invalid?5LOC?5header?5?$CIbad?5signatu@ 100103d0     zip_util.obj
 0002:000043f4       ??_C@_0BK@DBEMIBFN@ZIP_Read?3?5jzentry?5is?5NULL@ 100103f4     zip_util.obj
 0002:00004410       ??_C@_0CI@IPMMKOEL@ZIP_Read?3?5specified?5offset?5out?5@ 10010410     zip_util.obj
 0002:00004438       ??_C@_0CP@NKNCEDJJ@ZIP_Read?3?5corrupt?5zip?5file?3?5inv@ 10010438     zip_util.obj
 0002:00004468       ??_C@_0CB@CIEAIEG@ZIP_Read?3?5error?5reading?5zip?5fil@ 10010468     zip_util.obj
 0002:0000448c       ??_C@_0CD@NHPFPCNC@inflateFully?3?5entry?5not?5compres@ 1001048c     zip_util.obj
 0002:000044b0       ??_C@_0CF@CIDJLPNC@inflateFully?3?5Unexpected?5end?5of@ 100104b0     zip_util.obj
 0002:000044d8       ??_C@_0CH@CEOIBOIL@inflateFully?3?5Unexpected?5end?5of@ 100104d8     zip_util.obj
 0002:00004500       ??_C@_0BE@OKLOKMGK@jzentry?5was?5invalid@ 10010500     zip_util.obj
 0002:00004514       ??_C@_07KJFPOMFC@?$CFs?3?5?$CFs?6@ 10010514     zip_util.obj
 0002:0000451c       ??_C@_0DA@PDLLELGI@INFLATER_inflateFully?3?5Unexpect@ 1001051c     zip_util.obj
 0002:0000454c       ??_C@_0DB@FKHEPCI@INFLATER_inflateFully?3?5Compress@ 1001054c     zip_util.obj
 0002:00004580       ??_C@_0CF@BBAHGKKG@INFLATER_inflateFully?3?5out?5of?5m@ 10010580     zip_util.obj
 0002:000045a8       ??_C@_0CG@IIFAIDPA@INFLATER_inflateFully?3?5internal@ 100105a8     zip_util.obj
 0002:000045d0       ??_C@_0BO@DIJIDOL@Out?5of?5memory?5in?5deflateInit2@ 100105d0     zip_util.obj
 0002:000045f0       ??_C@_0BP@DLMACEHJ@Internal?5error?5in?5deflateInit2@ 100105f0     zip_util.obj
 0002:00004610       ??_C@_0BB@OLKJDAH@Buffer?5too?5small@ 10010610     zip_util.obj
 0002:00004624       ??_C@_0BF@OOJIEEPG@Intern?5deflate?5error@ 10010624     zip_util.obj
 0002:0000463c       _z_errmsg                  1001063c     zutil.obj
 0002:00004664       ??_C@_0BA@MOKMMFOD@need?5dictionary@ 10010664     zutil.obj
 0002:00004674       ??_C@_0L@FNAOCBOG@stream?5end@ 10010674     zutil.obj
 0002:00004680       ??_C@_0L@KIJFAKBJ@file?5error@ 10010680     zutil.obj
 0002:0000468c       ??_C@_0N@MKKNPMJD@stream?5error@ 1001068c     zutil.obj
 0002:0000469c       ??_C@_0L@HAHMBNLP@data?5error@ 1001069c     zutil.obj
 0002:000046a8       ??_C@_0BE@OGGJBMCE@insufficient?5memory@ 100106a8     zutil.obj
 0002:000046bc       ??_C@_0N@DFPGLBGC@buffer?5error@ 100106bc     zutil.obj
 0002:000046cc       ??_C@_0BF@CJFPCCEG@incompatible?5version@ 100106cc     zutil.obj
 0002:000046e4       __pRawDllMain              100106e4     MSVCRT:dll_dllmain.obj
 0002:000046e4       __pDefaultRawDllMain       100106e4     MSVCRT:dll_dllmain.obj
 0002:00004760       __load_config_used         10010760     MSVCRT:loadcfg.obj
 0002:00004818       ___safe_se_handler_table   10010818     <linker-defined>
 0002:00004a9c       ___rtc_iaa                 10010a9c     MSVCRT:initsect.obj
 0002:00004aa0       ___rtc_izz                 10010aa0     MSVCRT:initsect.obj
 0002:00004aa4       ___rtc_taa                 10010aa4     MSVCRT:initsect.obj
 0002:00004aa8       ___rtc_tzz                 10010aa8     MSVCRT:initsect.obj
 0002:00005208       __IMPORT_DESCRIPTOR_jvm    10011208     jvm:jvm.dll
 0002:0000521c       __IMPORT_DESCRIPTOR_java   1001121c     java:java.dll
 0002:00005230       __IMPORT_DESCRIPTOR_KERNEL32 10011230     kernel32:KERNEL32.dll
 0002:00005244       __IMPORT_DESCRIPTOR_VCRUNTIME140 10011244     vcruntime:VCRUNTIME140.dll
 0002:00005258       __IMPORT_DESCRIPTOR_api-ms-win-crt-heap-l1-1-0 10011258     ucrt:api-ms-win-crt-heap-l1-1-0.dll
 0002:0000526c       __IMPORT_DESCRIPTOR_api-ms-win-crt-stdio-l1-1-0 1001126c     ucrt:api-ms-win-crt-stdio-l1-1-0.dll
 0002:00005280       __IMPORT_DESCRIPTOR_api-ms-win-crt-string-l1-1-0 10011280     ucrt:api-ms-win-crt-string-l1-1-0.dll
 0002:00005294       __IMPORT_DESCRIPTOR_api-ms-win-crt-runtime-l1-1-0 10011294     ucrt:api-ms-win-crt-runtime-l1-1-0.dll
 0002:000052a8       __NULL_IMPORT_DESCRIPTOR   100112a8     jvm:jvm.dll
 0003:00000004       ___security_cookie_complement 10012004     MSVCRT:gs_cookie.obj
 0003:00000008       ___security_cookie         10012008     MSVCRT:gs_cookie.obj
 0003:00000010       ___scrt_native_dllmain_reason 10012010     MSVCRT:utility.obj
 0003:00000020       ___isa_enabled             10012020     MSVCRT:cpu_disp.obj
 0003:00000024       ___scrt_ucrt_dll_is_in_use 10012024     MSVCRT:ucrt_stubs.obj
 0003:00000360       ?__type_info_root_node@@3U__type_info_node@@A 10012360     MSVCRT:tncleanup.obj
 0003:00000368       ?_OptionsStorage@?1??__local_stdio_scanf_options@@9@4_KA 10012368     MSVCRT:default_local_stdio_options.obj
 0003:00000370       ___scrt_current_native_startup_state 10012370     MSVCRT:utility.obj
 0003:00000374       ___scrt_native_startup_lock 10012374     MSVCRT:utility.obj
 0003:00000394       ___scrt_debugger_hook_flag 10012394     MSVCRT:utility_desktop.obj
 0003:00000398       ___isa_available           10012398     MSVCRT:cpu_disp.obj
 0003:0000039c       ___favor                   1001239c     MSVCRT:cpu_disp.obj
 0003:000003a0       ?_OptionsStorage@?1??__local_stdio_printf_options@@9@9 100123a0     <common>
 0003:000003a8       ___dyn_tls_init_callback   100123a8     <common>

 entry point at        0001:0000965d

 Static symbols

 0000:fffeb000       .debug$S                   10000000     zip.exp
 0000:fffeb000       .debug$S                   10000000     vcruntime:VCRUNTIME140.dll
 0000:fffeb000       .debug$S                   10000000     vcruntime:VCRUNTIME140.dll
 0000:fffeb000       .debug$S                   10000000     vcruntime:VCRUNTIME140.dll
 0000:fffeb000       .debug$S                   10000000     vcruntime:VCRUNTIME140.dll
 0000:fffeb000       .debug$S                   10000000     vcruntime:VCRUNTIME140.dll
 0000:fffeb000       .debug$S                   10000000     vcruntime:VCRUNTIME140.dll
 0000:fffeb000       .debug$S                   10000000     vcruntime:VCRUNTIME140.dll
 0000:fffeb000       .debug$S                   10000000     ucrt:api-ms-win-crt-convert-l1-1-0.dll
 0002:ffff4000       .idata$6                   10000000     ucrt:api-ms-win-crt-convert-l1-1-0.dll
 0000:fffeb000       .debug$S                   10000000     ucrt:api-ms-win-crt-heap-l1-1-0.dll
 0000:fffeb000       .debug$S                   10000000     ucrt:api-ms-win-crt-heap-l1-1-0.dll
 0000:fffeb000       .debug$S                   10000000     ucrt:api-ms-win-crt-heap-l1-1-0.dll
 0000:fffeb000       .debug$S                   10000000     ucrt:api-ms-win-crt-heap-l1-1-0.dll
 0000:fffeb000       .debug$S                   10000000     ucrt:api-ms-win-crt-runtime-l1-1-0.dll
 0000:fffeb000       .debug$S                   10000000     ucrt:api-ms-win-crt-runtime-l1-1-0.dll
 0000:fffeb000       .debug$S                   10000000     ucrt:api-ms-win-crt-runtime-l1-1-0.dll
 0000:fffeb000       .debug$S                   10000000     ucrt:api-ms-win-crt-runtime-l1-1-0.dll
 0000:fffeb000       .debug$S                   10000000     ucrt:api-ms-win-crt-runtime-l1-1-0.dll
 0000:fffeb000       .debug$S                   10000000     ucrt:api-ms-win-crt-runtime-l1-1-0.dll
 0000:fffeb000       .debug$S                   10000000     ucrt:api-ms-win-crt-runtime-l1-1-0.dll
 0000:fffeb000       .debug$S                   10000000     ucrt:api-ms-win-crt-runtime-l1-1-0.dll
 0000:fffeb000       .debug$S                   10000000     ucrt:api-ms-win-crt-runtime-l1-1-0.dll
 0000:fffeb000       .debug$S                   10000000     ucrt:api-ms-win-crt-runtime-l1-1-0.dll
 0000:fffeb000       .debug$S                   10000000     ucrt:api-ms-win-crt-runtime-l1-1-0.dll
 0000:fffeb000       .debug$S                   10000000     ucrt:api-ms-win-crt-runtime-l1-1-0.dll
 0000:fffeb000       .debug$S                   10000000     ucrt:api-ms-win-crt-runtime-l1-1-0.dll
 0000:fffeb000       .debug$S                   10000000     ucrt:api-ms-win-crt-runtime-l1-1-0.dll
 0000:fffeb000       .debug$S                   10000000     ucrt:api-ms-win-crt-stdio-l1-1-0.dll
 0000:fffeb000       .debug$S                   10000000     ucrt:api-ms-win-crt-stdio-l1-1-0.dll
 0000:fffeb000       .debug$S                   10000000     ucrt:api-ms-win-crt-stdio-l1-1-0.dll
 0000:fffeb000       .debug$S                   10000000     ucrt:api-ms-win-crt-stdio-l1-1-0.dll
 0000:fffeb000       .debug$S                   10000000     ucrt:api-ms-win-crt-stdio-l1-1-0.dll
 0000:fffeb000       .debug$S                   10000000     ucrt:api-ms-win-crt-stdio-l1-1-0.dll
 0000:fffeb000       .debug$S                   10000000     ucrt:api-ms-win-crt-stdio-l1-1-0.dll
 0000:fffeb000       .debug$S                   10000000     ucrt:api-ms-win-crt-stdio-l1-1-0.dll
 0000:fffeb000       .debug$S                   10000000     ucrt:api-ms-win-crt-string-l1-1-0.dll
 0000:fffeb000       .debug$S                   10000000     ucrt:api-ms-win-crt-string-l1-1-0.dll
 0000:fffeb000       .debug$S                   10000000     ucrt:api-ms-win-crt-string-l1-1-0.dll
 0000:fffeb000       .debug$S                   10000000     ucrt:api-ms-win-crt-string-l1-1-0.dll
 0000:fffeb000       .debug$S                   10000000     kernel32:KERNEL32.dll
 0000:fffeb000       .debug$S                   10000000     kernel32:KERNEL32.dll
 0000:fffeb000       .debug$S                   10000000     kernel32:KERNEL32.dll
 0000:fffeb000       .debug$S                   10000000     kernel32:KERNEL32.dll
 0000:fffeb000       .debug$S                   10000000     kernel32:KERNEL32.dll
 0000:fffeb000       .debug$S                   10000000     kernel32:KERNEL32.dll
 0000:fffeb000       .debug$S                   10000000     kernel32:KERNEL32.dll
 0000:fffeb000       .debug$S                   10000000     kernel32:KERNEL32.dll
 0000:fffeb000       .debug$S                   10000000     kernel32:KERNEL32.dll
 0000:fffeb000       .debug$S                   10000000     kernel32:KERNEL32.dll
 0000:fffeb000       .debug$S                   10000000     kernel32:KERNEL32.dll
 0000:fffeb000       .debug$S                   10000000     kernel32:KERNEL32.dll
 0000:fffeb000       .debug$S                   10000000     kernel32:KERNEL32.dll
 0000:fffeb000       .debug$S                   10000000     kernel32:KERNEL32.dll
 0000:fffeb000       .debug$S                   10000000     kernel32:KERNEL32.dll
 0000:fffeb000       .debug$S                   10000000     kernel32:KERNEL32.dll
 0000:fffeb000       .debug$S                   10000000     kernel32:KERNEL32.dll
 0000:fffeb000       .debug$S                   10000000     kernel32:KERNEL32.dll
 0000:fffeb000       .debug$S                   10000000     jvm:jvm.dll
 0000:fffeb000       .debug$S                   10000000     jvm:jvm.dll
 0000:fffeb000       .debug$S                   10000000     jvm:jvm.dll
 0000:fffeb000       .debug$S                   10000000     jvm:jvm.dll
 0000:fffeb000       .debug$S                   10000000     jvm:jvm.dll
 0000:fffeb000       .debug$S                   10000000     jvm:jvm.dll
 0000:fffeb000       .debug$S                   10000000     java:java.dll
 0000:fffeb000       .debug$S                   10000000     java:java.dll
 0000:fffeb000       .debug$S                   10000000     java:java.dll
 0000:fffeb000       .debug$S                   10000000     java:java.dll
 0000:fffeb000       .debug$S                   10000000     java:java.dll
 0000:fffeb000       .debug$S                   10000000     java:java.dll
 0000:fffeb000       .debug$S                   10000000     java:java.dll
 0000:fffeb000       .debug$S                   10000000     java:java.dll
 0000:fffeb000       .debug$S                   10000000     java:java.dll
 0001:000004ed       _checkDeflateStatus        100014ed f   Deflater.obj
 0001:000005a2       _checkSetDictionaryResult  100015a2 f   Deflater.obj
 0001:000005d2       _doDeflate                 100015d2 f   Deflater.obj
 0001:0000061b       _throwInternalErrorHelper  1000161b f   Deflater.obj
 0001:000009e9       _checkInflateStatus        100019e9 f   Inflater.obj
 0001:00000b28       _checkSetDictionaryResult  10001b28 f   Inflater.obj
 0001:00000b5c       _doInflate                 10001b5c f   Inflater.obj
 0001:00000b85       _deflate_stored            10001b85 f   deflate.obj
 0001:00000eed       _deflate_fast              10001eed f   deflate.obj
 0001:00001229       _deflate_slow              10002229 f   deflate.obj
 0001:0000258e       _deflateStateCheck         1000358e f   deflate.obj
 0001:000025e1       _deflate_huff              100035e1 f   deflate.obj
 0001:00002745       _deflate_rle               10003745 f   deflate.obj
 0001:000029d5       _fill_window               100039d5 f   deflate.obj
 0001:00002b6d       _flush_pending             10003b6d f   deflate.obj
 0001:00002bb6       _lm_init                   10003bb6 f   deflate.obj
 0001:00002c43       _longest_match             10003c43 f   deflate.obj
 0001:00002dad       _putShortMSB               10003dad f   deflate.obj
 0001:00002dd7       _read_buf                  10003dd7 f   deflate.obj
 0001:00002e41       _slide_hash                10003e41 f   deflate.obj
 0001:0000493e       $LN759                     1000593e     inflate.obj
 0001:00004c29       _inflateStateCheck         10005c29 f   inflate.obj
 0001:00004c5c       _updatewindow              10005c5c f   inflate.obj
 0001:00005569       _bi_flush                  10006569 f   trees.obj
 0001:000055d5       _bi_windup                 100065d5 f   trees.obj
 0001:0000562c       _build_bl_tree             1000662c f   trees.obj
 0001:00005692       _build_tree                10006692 f   trees.obj
 0001:00005922       _compress_block            10006922 f   trees.obj
 0001:00005d03       _detect_data_type          10006d03 f   trees.obj
 0001:00005d6b       _gen_bitlen                10006d6b f   trees.obj
 0001:00005f87       _init_block                10006f87 f   trees.obj
 0001:00005ff6       _pqdownheap                10006ff6 f   trees.obj
 0001:000060ad       _scan_tree                 100070ad f   trees.obj
 0001:00006189       _send_all_trees            10007189 f   trees.obj
 0001:000063e5       _send_tree                 100073e5 f   trees.obj
 0001:00006afb       _crc32_little              10007afb f   zcrc32.obj
 0001:00006f61       _ZFILE_Open                10007f61 f   zip_util.obj
 0001:00007c20       _addMetaName               10008c20 f   zip_util.obj
 0001:00007ca5       _countCENHeaders           10008ca5 f   zip_util.obj
 0001:00007d07       _deflateInit2Wrapper       10008d07 f   zip_util.obj
 0001:00007d7c       _findEND                   10008d7c f   zip_util.obj
 0001:00007fe3       _findEND64                 10008fe3 f   zip_util.obj
 0001:000080ab       _freeCEN                   100090ab f   zip_util.obj
 0001:000080f9       _freeZip                   100090f9 f   zip_util.obj
 0001:00008156       _growMetaNames             10009156 f   zip_util.obj
 0001:0000819f       _hashN                     1000919f f   zip_util.obj
 0001:000081be       _newEntry                  100091be f   zip_util.obj
 0001:000087e3       _readCEN                   100097e3 f   zip_util.obj
 0001:00008d42       _readCENHeader             10009d42 f   zip_util.obj
 0001:00008e1e       _readFully                 10009e1e f   zip_util.obj
 0001:00008e88       _readFullyAt               10009e88 f   zip_util.obj
 0001:00008ec2       _sequentialAccessReadCENHeader 10009ec2 f   zip_util.obj
 0001:00008fed       _tracking_zlib_alloc       10009fed f   zip_util.obj
 0001:0000900c       _tracking_zlib_free        1000a00c f   zip_util.obj
 0001:00009018       _verifyEND                 1000a018 f   zip_util.obj
 0001:0000917e       _zlib_block_alloc          1000a17e f   zip_util.obj
 0001:000091a5       _zlib_block_free           1000a1a5 f   zip_util.obj
 0001:00009230       $$000000                   1000a230     MSVCRT:llrem.obj
 0001:000092f0       $$000000                   1000a2f0     MSVCRT:chkstk.obj
 0001:0000931d       ?dllmain_crt_dispatch@@YGHQAUHINSTANCE__@@KQAX@Z 1000a31d f   MSVCRT:dll_dllmain.obj
 0001:00009370       ?dllmain_crt_process_attach@@YAHQAUHINSTANCE__@@QAX@Z 1000a370 f   MSVCRT:dll_dllmain.obj
 0001:00009477       ?dllmain_crt_process_detach@@YAH_N@Z 1000a477 f   MSVCRT:dll_dllmain.obj
 0001:00009527       ?dllmain_dispatch@@YAHQAUHINSTANCE__@@KQAX@Z 1000a527 f   MSVCRT:dll_dllmain.obj
 0001:00009632       ?dllmain_raw@@YGHQAUHINSTANCE__@@KQAX@Z 1000a632 f   MSVCRT:dll_dllmain.obj
 0001:000097a1       ___get_entropy             1000a7a1 f   MSVCRT:gs_support.obj
 0001:00009896       ?find_pe_section@@YAPAU_IMAGE_SECTION_HEADER@@QAEI@Z 1000a896 f   MSVCRT:utility.obj
 0001:00009cf0       $$000000                   1000acf0     MSVCRT:sehprolg4.obj
 0002:00000300       _configuration_table       1000c300     deflate.obj
 0002:00000378       ?my_version@?1??deflateInit2_@@9@9 1000c378     deflate.obj
 0002:00000380       ?lenfix@?1??fixedtables@@9@9 1000c380     infback.obj
 0002:00000b80       ?distfix@?1??fixedtables@@9@9 1000cb80     infback.obj
 0002:00000c00       ?order@?1??inflateBack@@9@9 1000cc00     infback.obj
 0002:00000d68       ?lenfix@?1??fixedtables@@9@9 1000cd68     inflate.obj
 0002:00001568       ?distfix@?1??fixedtables@@9@9 1000d568     inflate.obj
 0002:000015e8       ?order@?1??inflate@@9@9    1000d5e8     inflate.obj
 0002:000016e8       ?lbase@?1??inflate_table@@9@9 1000d6e8     inftrees.obj
 0002:00001728       ?lext@?1??inflate_table@@9@9 1000d728     inftrees.obj
 0002:00001768       ?dbase@?1??inflate_table@@9@9 1000d768     inftrees.obj
 0002:000017a8       ?dext@?1??inflate_table@@9@9 1000d7a8     inftrees.obj
 0002:00001ae8       _extra_lbits               1000dae8     trees.obj
 0002:00001b5c       _bl_order                  1000db5c     trees.obj
 0002:00001b70       _extra_dbits               1000db70     trees.obj
 0002:00001be8       _extra_blbits              1000dbe8     trees.obj
 0002:00001c38       _static_ltree              1000dc38     trees.obj
 0002:000020b8       _static_dtree              1000e0b8     trees.obj
 0002:00002130       _base_length               1000e130     trees.obj
 0002:000021a8       _base_dist                 1000e1a8     trees.obj
 0002:00002220       _static_l_desc             1000e220     trees.obj
 0002:00002234       _static_d_desc             1000e234     trees.obj
 0002:00002248       _static_bl_desc            1000e248     trees.obj
 0002:00002260       _crc_table                 1000e260     zcrc32.obj
 0002:00004260       _END_MAXLEN                10010260     zip_util.obj
 0002:000046e8       _GS_ExceptionPointers      100106e8     MSVCRT:gs_report.obj
 0002:00004ab0       __sehtable$?dllmain_crt_process_attach@@YAHQAUHINSTANCE__@@QAX@Z 10010ab0     MSVCRT:dll_dllmain.obj
 0002:00004ad0       __sehtable$?dllmain_crt_process_detach@@YAH_N@Z 10010ad0     MSVCRT:dll_dllmain.obj
 0002:00004af8       __sehtable$?dllmain_dispatch@@YAHQAUHINSTANCE__@@KQAX@Z 10010af8     MSVCRT:dll_dllmain.obj
 0002:00004b18       __sehtable$___scrt_is_nonwritable_in_current_image 10010b18     MSVCRT:utility.obj
 0002:00004b40       .edata                     10010b40     zip.exp
 0002:00004b68       rgpv                       10010b68     zip.exp
 0002:00004bf8       rgszName                   10010bf8     zip.exp
 0002:00004c88       rgwOrd                     10010c88     zip.exp
 0002:00004cd0       szName                     10010cd0     zip.exp
 0002:00004cd8       $N00001                    10010cd8     zip.exp
 0002:00004cfe       $N00002                    10010cfe     zip.exp
 0002:00004d2e       $N00003                    10010d2e     zip.exp
 0002:00004d59       $N00004                    10010d59     zip.exp
 0002:00004d7d       $N00005                    10010d7d     zip.exp
 0002:00004dac       $N00006                    10010dac     zip.exp
 0002:00004dd6       $N00007                    10010dd6     zip.exp
 0002:00004e0a       $N00008                    10010e0a     zip.exp
 0002:00004e3d       $N00009                    10010e3d     zip.exp
 0002:00004e70       $N00010                    10010e70     zip.exp
 0002:00004ea2       $N00011                    10010ea2     zip.exp
 0002:00004ec6       $N00012                    10010ec6     zip.exp
 0002:00004eef       $N00013                    10010eef     zip.exp
 0002:00004f14       $N00014                    10010f14     zip.exp
 0002:00004f3a       $N00015                    10010f3a     zip.exp
 0002:00004f68       $N00016                    10010f68     zip.exp
 0002:00004f9c       $N00017                    10010f9c     zip.exp
 0002:00004fc0       $N00018                    10010fc0     zip.exp
 0002:00004fe9       $N00019                    10010fe9     zip.exp
 0002:0000501d       $N00020                    1001101d     zip.exp
 0002:00005050       $N00021                    10011050     zip.exp
 0002:00005083       $N00022                    10011083     zip.exp
 0002:000050b5       $N00023                    100110b5     zip.exp
 0002:000050da       $N00024                    100110da     zip.exp
 0002:00005101       $N00025                    10011101     zip.exp
 0002:00005127       $N00026                    10011127     zip.exp
 0002:00005155       $N00027                    10011155     zip.exp
 0002:00005189       $N00028                    10011189     zip.exp
 0002:00005193       $N00029                    10011193     zip.exp
 0002:0000519d       $N00030                    1001119d     zip.exp
 0002:000051ab       $N00031                    100111ab     zip.exp
 0002:000051ba       $N00032                    100111ba     zip.exp
 0002:000051ce       $N00033                    100111ce     zip.exp
 0002:000051df       $N00034                    100111df     zip.exp
 0002:000051f0       $N00035                    100111f0     zip.exp
 0002:000051f9       $N00036                    100111f9     zip.exp
 0002:0000543a       .idata$6                   1001143a     jvm:jvm.dll
 0002:00005518       .idata$6                   10011518     java:java.dll
 0002:00005686       .idata$6                   10011686     kernel32:KERNEL32.dll
 0002:000056e2       .idata$6                   100116e2     vcruntime:VCRUNTIME140.dll
 0002:00005804       .idata$6                   10011804     ucrt:api-ms-win-crt-heap-l1-1-0.dll
 0002:00005824       .idata$6                   10011824     ucrt:api-ms-win-crt-stdio-l1-1-0.dll
 0002:00005844       .idata$6                   10011844     ucrt:api-ms-win-crt-string-l1-1-0.dll
 0002:00005866       .idata$6                   10011866     ucrt:api-ms-win-crt-runtime-l1-1-0.dll
 0003:00000000       _INITIAL_META_COUNT        10012000     zip_util.obj
 0003:00000028       _inputConsumedID           10012028     Inflater.obj
 0003:0000002c       _outputConsumedID          1001202c     Inflater.obj
 0003:00000030       _zfiles                    10012030     zip_util.obj
 0003:00000034       _zfiles_lock               10012034     zip_util.obj
 0003:00000038       ?inited@?1??InitializeZip@@9@9 10012038     zip_util.obj
 0003:0000003c       ?__proc_attached@@3HA      1001203c     MSVCRT:dll_dllmain.obj
 0003:00000040       _GS_ExceptionRecord        10012040     MSVCRT:gs_report.obj
 0003:00000090       _GS_ContextRecord          10012090     MSVCRT:gs_report.obj
 0003:00000378       ?is_initialized_as_dll@@3_NA 10012378     MSVCRT:utility.obj
 0003:00000379       ?module_local_atexit_table_initialized@@3_NA 10012379     MSVCRT:utility.obj
 0003:0000037c       ?module_local_atexit_table@@3U_onexit_table_t@@A 1001237c     MSVCRT:utility.obj
 0003:00000388       ?module_local_at_quick_exit_table@@3U_onexit_table_t@@A 10012388     MSVCRT:utility.obj
 0004:00000060       $R000000                   10013060     zip.dll.res
